:1000000001308A00A729000085100510831685108D
:1000100005101F169F121F1783129F171F141F13FF
:1000200083161F109F101F159F1108308312C100E7
:100030001F08E33941049F0085128316851283123D
:10004000B4294F3084000008031934280130C1005E
:10005000C001C00B2928C10B28284A30C000C00BA2
:100060002F283228800B262808009F1450109F1C30
:10007000501450183F2850109F1C501439289F18B6
:100080003F281E08C30083161E088312D1001E08D5
:10009000D2005108C1005208C200080035204208B1
:1000A000CF004108CE0035204108CE074208031892
:1000B000420FCF0735204108CE0742080318420FF0
:1000C000CF0735204108CE0742080318420FCF075B
:1000D00035204108CE0742080318420FCF073520CC
:1000E0004108CE0742080318420FCF0735204108C8
:1000F000CE0742080318420FCF0735204108CE072C
:1001000042080318420FCF0735204108CE074208A6
:100110000318420FCF0735204108CE0742080318C5
:10012000420FCF0735204108CE0742080318420F7F
:10013000CF0735204108CE0742080318420FCF07EA
:1001400035204108CE0742080318420FCF0735205B
:100150004108CE0742080318420FCF073520410857
:10016000CE0742080318420FCF0735204108CE07BB
:1001700042080318420FCF074F0CC3004E0CC200B9
:10018000C30CC20CC30CC20CC30CC20C0F30C30591
:100190004208C1004308C200080035204208CF00D1
:1001A0004108CE0035204108CE0742080318420F0F
:1001B000CF0735204208C3004108CE074208031884
:1001C000420FCF0735204108CE0742080318420FDF
:1001D000CF074F0CC3004E0CC200C30CC20C3F3003
:1001E000C3054208C1004308C20008008E30C000A9
:1001F0004F08C1004E08C200C301C108031D0A29EF
:100200004208C100C2010830C002C108031D0A290A
:10021000C00112290310C11B1129C20DC10DC00359
:100220000A29C11308004E0803198329D600520871
:1002300003198329D607031824297F30D602031C0B
:1002400083290319832928298130D6070318832994
:100250005608C000C101C201C3014F08DA00DA1715
:100260005008D9005108D8001830D600D701581CC2
:1002700051295508C307031C4329C20A031D4329FA
:10028000C10A0319D7175408C207031C4A29C10A17
:100290000319D7175308D000D0175008C107031807
:1002A000D717D70DC10CC20CC30CDA0CD90CD80C63
:1002B0000310D60B36290130C00703188329C11B50
:1002C0006829DA0DC30DC20DC10DC00303198329BE
:1002D000DA1F7929C30A031D7929C20A031D792966
:1002E000C10A031D7929C10CC20CC30CC00A031931
:1002F00083294F08D7005308D706D71F8129C11774
:100300008729C1138729C001C101C201C3010800A7
:100310008E30C0004E08C0024F08C2005008C10015
:10032000C217C00803199F290310C208031D9B2987
:10033000C10803199F29C20CC10CC00B9429CF1FFF
:10034000A629C109C209C10A0319C20A0800840109
:100350001F3083051F1383161F109F101F119F113D
:1003600083129A019C0104286430CF0021204E2082
:100370004208CF004108CE004F08013C031CC829A9
:10038000031DC6294E08053C031CC8298A01002804
:100390000730CE00C830CF002120CE0BCA2905146B
:1003A0000230CE00FA30CF002120CE0BD229CD2052
:1003B0004208C5004108C4004508CF004408CE00EB
:1003C000F6204308D1004208D0004108CF00400881
:1003D000CE003330D500D400D3007E30D2001321BC
:1003E0004308D1004208D0004108CF004008CE00A9
:1003F00088214208C7004108C600051A8514CD208F
:100400004208CF004108CE0047084F02031C142ABF
:10041000031D0E2A4E0846020318142A051A122A32
:100420008510132A8514FF2985103230CF00212032
:1004300005100330CB00FF30CA000330C900FF3085
:10044000C80085164E204208CB004108CA004E2045
:100450004208CD004108CC004D084B02031C5C2A29
:10046000031D362A4A084C0203185C2A4D08CB00AB
:100470004C08CA004B08CF004A08CE00F6204308BB
:10048000D1004208D0004108CF004008CE006630BD
:10049000D500D4000630D3007F30D20013214308AA
:1004A000D1004208D0004108CF004008CE0088218A
:1004B0004208C9004108C80049084D02031C6C2AC3
:1004C000031D662A4C08480203186C2A83168514FB
:1004D00005148A01831200284D08013C031C802A60
:1004E000031D762A4C08053C031C802A83168514BC
:1004F0000514831285126430CF0021208A01002860
:0A0500000A30CF002120272A6300F3
:02400E00043F6D
:00000001FF
